:100000000C94EC020C9424030C9424030C9424030D
:100010000C9424030C9424030C9424030C942403C4
:100020000C9424030C9424030C94C7280C94992951
:100030000C94A6230C9424030C9424030C94240302
:100040000C9424030C9424030C9424030C94240394
:100050000C9424030C942E240C9424030C94240359
:100060000C9424030C9424030C9424030C94240374
:100070000C9424030C9424030C9424030C94240364
:100080000C9424030C9424030C9424030C94240354
:100090000C9424030C9424030C9424030C94240344
:1000A0000C9424030C9424030C9424038B068B06D9
:1000B000B706B7061F073D07550855084807E1076B
:1000C000F207F207062A2D2A252B2D2A252B792A1D
:1000D0009C2A252BF32A022B290014001A00080061
:1000E000150017001C0018000C00120013002A0055
:1000F0002B0004001600070009000A000B000D0089
:100100000E000F0000002800E10000001D001B0091
:1001100006001900050011001000360037003800F5
:10012000E000E300E20000002C412C42000000004F
:100130000000E343E600E40035021E021F02200235
:1001400021022202230224022502260227022A007B
:100150003A003B003C003D003E003F002D022E02D5
:100160002F02300200003102400000004100420036
:1001700043004400450032026402C05CBF5CBE5CC8
:10018000010001000100000001005000000000001B
:100190000000510052004F0035001E001F002000DB
:1001A00021002200230024002500260027002A0029
:1001B0003A003B003C003D003E003F002D002E0079
:1001C0002F003000000031004000000041004200DC
:1001D00043004400450032006400010001004C006F
:1001E000010001000100000001000100000000000A
:1001F000000001000100C35C0100005C010001007F
:1002000001000100010001000100010001004C009B
:100210000100010001001D5C1E5C135C0A5C010012
:1002200001000100000001000100000001000100C8
:10023000C35CC45CC65CC75CC85CC95CCA5CCB5CA4
:10024000A600010001000000010001000000000004
:10025000000001000100010000047F3F1F64321410
:10026000643214783C1E1E140A05222325262829F0
:100270002A2C2D2F3032333536383A3B3D3E404222
:10028000434547494A4C4E5051535557595A5C5E65
:100290006062646668696B6D6F71737577797B7D79
:1002A0007F81838587898A8C8E90929496989A9C78
:1002B0009E9FA1A3A5A7A8AAACAEAFB1B3B4B6B890
:1002C000B9BBBCBEBFC1C2C3C5C6C7C9CACBCCCDF2
:1002D000CED0D1D2D2D3D4D5D6D7D7D8D9D9DADACD
:1002E000DBDBDBDCDCDCDCDCDDDDDDDDDCDCDCDC4D
:1002F000DCDBDBDBDADAD9D9D8D7D7D6D5D4D3D281
:10030000D2D1D0CECDCCCBCAC9C7C6C5C3C2C1BF5E
:10031000BEBCBBB9B8B6B4B3B1AFAEACAAA8A7A5C2
:10032000A3A19F9E9C9A98969492908E8C8A89877E
:100330008583817F7D7B79777573716F6D6B69685C
:10034000666462605E5C5A5957555351504E4C4A30
:100350004947454342403E3D3B3A383635333230DB
:100360002F2D2C2A292826252322FFAA7F5540003D
:100370000101010101010101010202020202020266
:100380000202030303030303030304040404040439
:1003900004050505050506060606060707070707FF
:1003A00008080808090909090A0A0A0B0B0B0C0CB2
:1003B0000C0D0D0D0E0E0E0F0F0F1010111111124E
:1003C0001213131414151516161717181819191ACD
:1003D0001A1B1B1C1D1D1E1E1F2020212222232430
:1003E00024252626272829292A2B2C2D2D2E2F306F
:1003F000313232333435363738393A3B3C3D3E3F83
:10040000404142434445464748494A4C4D4E4F506F
:10041000515354555658595A5B5D5E5F616264652D
:100420006668696B6C6D6F7072737577787A7B7DB7
:100430007E8082838587888A8C8E8F91939596980B
:100440009A9C9EA0A2A3A5A7A9ABADAFB1B3B5B727
:10045000BABCBEC0C2C4C6C9CBCDCFD1D4D6D8DBFE
:10046000DDDFE2E4E7E9EBEEF0F3F5F8FAFDFF0C8F
:100470000341004D004A00340030000000120348E0
:100480000061006E0020004300680065006E0000FF
:10049000000403090409023B00020100A0FA090458
:1004A00000000103010100092111010001224000A7
:1004B0000705810308000109040100010300000091
:1004C00009211101000122B6000705820320000165
:1004D0001201000200000008EDFE7260020001023D
:1004E000000105010902A10185020901A100050918
:1004F00019012908150025019508750181020501DA
:10050000093009311581257F950275088106093862
:100510001581257F950175088106050C0A3802159D
:1005200081257F950175088106C0C005010980A15C
:1005300001850319012AB700150126B70095017539
:10054000108100C0050C0901A101850419012AA030
:1005500002150126A002950175108100C005010950
:1005600006A1018506050719E029E7150025019573
:1005700008750181020507190029EF15002501956D
:10058000F07501810205081901290595057501918C
:1005900002950175039101C005010906A101050736
:1005A00019E029E7150025019508750181029501DB
:1005B000750881010507190029FF150026FF009520
:1005C0000675088100050819012905950575019131
:1005D00002950175039101C011241FBECFEFDAE02F
:1005E000DEBFCDBF04B603FE18C08091FD0290911E
:1005F000FE02A091FF02B09100038730904BA7400C
:10060000B04B59F41092FD021092FE021092FF02BC
:1006100010920003E0E0F8E3099511E0A0E0B1E0FA
:10062000ECE9F8E502C005900D92A43CB107D9F7BA
:1006300022E0A4ECB1E001C01D92AD3FB207E1F7AA
:100640000E9467140C944C2C0C940000CF93FB0177
:10065000893A2DE5920751F08A3A2DE59207D1F0BB
:10066000883A9D4511F5C28181E002C0C28182E0D5
:10067000CC2341F00E949D0943E062E081E00E94AA
:10068000FD030EC00E94BE0943E062E081E00E94CB
:10069000FD030CC0C28183E0CC2321F00E949D09A0
:1006A000C0E004C00E94BE0901C0C1E08C2FCF9100
:1006B000089581E008950C94260308950C945D0339
:1006C0001F93CF93DF9300D000D01F92CDB7DEB73A
:1006D00049835A836B833091C70189819A81311193
:1006E00014C0662359F0222349F00E94920A182F61
:1006F000682F89819A810E943B0A03C00E94660A82
:10070000182F69817A81812F04C00E94920A698121
:100710007A810F900F900F900F900F90DF91CF91F3
:100720001F910C94D211FC01262F408151816281CE
:10073000738184810C94600381E00895CF93DF93EB
:10074000EC0160E00E949303BE01DF91CF910C9415
:100750005E038F929F92AF92BF92CF92DF92EF9201
:10076000FF920F931F936B017C0181E090E0A0E06A
:10077000B0E04C015D0104C0880C991CAA1CBB1C94
:100780004A95D2F7AC01BD0104C0440F551F661F46
:10079000771F2A95D2F7482959296A297B2904C04D
:1007A000880F991FAA1FBB1F0A95D2F78A019B01C8
:1007B0000C211D212E213F2140175107620773078D
:1007C00039F4BC01CD016C297D298E299F290AC0ED
:1007D00080959095A095B095BC01CD016C217D21AF
:1007E0008E219F211F910F91FF90EF90DF90CF906E
:1007F000BF90AF909F908F9008950F93382F262F22
:100800006091E6017091E7018091E8019091E90122
:10081000042F432F0E94A9030F910C9477090C9485
:1008200018130C94141308950E94E5080E941304F1
:100830002FEF84E39CE0215080409040E1F700C01E
:1008400000000C9454240F931F93CF93DF938C01DB
:1008500061E00E949303EC01B8010E945B038823CE
:1008600009F44BC0B801CE010E94E41E882309F4AC
:1008700044C0B801CE010E94F1218823F1F1B801F2
:10088000CE010E9405208823C1F1B801CE010E944B
:100890004D21882391F1B801CE010E94281D8823A3
:1008A00061F1F8018281882309F1CB358DE5D80704
:1008B000C1F050F4C115FCE5DF0781F0CF3DDC4508
:1008C000A9F40E94C90F19C0CC35EDE5DE0761F02F
:1008D000CD35DD4559F40E940C0F08C00E94140468
:1008E0000CC00E94150F02C00E94180FC801DF91B2
:1008F000CF911F910F910C94590380E0DF91CF911C
:100900001F910F9108950E94882380E00E94191F73
:100910000C94AE040E94081E0E94B1040C948E2315
:1009200008950C94900481E00895CF93C82F0E94FD
:100930009304882329F0C1FD02C02A9A01C02A9895
:10094000CF910895229A2A9A0895CF93C82F0E9492
:1009500091048C2F0E949504CF91089580E00C940F
:10096000A5040E944D220C94A5040E944D22909152
:10097000C601891721F08093C6010C94A50408953F
:10098000CF93DF93CDB7DEB72B970FB6F894DEBFCA
:100990000FBECDBF4F83588769877A878B876111D8
:1009A0000E94580E9E012F5F3F4F86E0F901119281
:1009B0008A95E9F785E0FE013796D90101900D92FD
:1009C0008A95E1F789819A814C815D81452B31F0CF
:1009D0009F3F31F491E08F3F19F403C091E001C0D3
:1009E00090E090FF09C049815A816B817C818D81A3
:1009F0009E810E94790D05C0C9010E949C0381114E
:100A0000F2CF2B960FB6F894DEBF0FBECDBFDF91AD
:100A1000CF910895FC01808191810E94D40A0895AC
:100A2000CF93882309F4A4C0C82F8238C1F40E9450
:100A30004D2281FD9DC069E38091020190910301E7
:100A40000E9443230E947A0E2FEF81EE94E0215002
:100A500080409040E1F700C0000069E319C083388E
:100A600001F50E944D2280FD83C063E58091020163
:100A7000909103010E9443230E947A0E2FEF81EE92
:100A800094E0215080409040E1F700C0000063E511
:100A900080910201909103010E944E23CF910C940A
:100AA0007A0E8438C1F40E944D2282FD61C067E451
:100AB00080910201909103010E9443230E947A0ECB
:100AC0002FEF81EE94E0215080409040E1F700C08C
:100AD000000067E4DDCF8CEF8C0F813AD0F46C2FEF
:100AE00080910201909103010E94C322882349F062
:100AF0006C2F80910201909103010E944E230E946D
:100B00007A0E6C2F80910201909103010E94432381
:100B1000C5CF80E28C0F883048F4C77081E001C0F7
:100B2000880FCA95EAF70E943B0EB8CFEBE5EC0FB1
:100B3000E33040F4F0E0E65AFE4F808190E0CF9140
:100B40000C948122E8E5EC0FE73150F4F0E0EE0F71
:100B5000FF1FE45DFE4F80819181CF910C9497221D
:100B6000CD3E30F08C2F0E94EC14CF910C94BE152A
:100B7000CF910895882309F464C0823879F40E94E3
:100B80004D2281FF5EC069E38091020190910301D3
:100B90000E9443230E947A0E69E310C08338B1F4A7
:100BA0000E944D2280FF4DC063E58091020190912B
:100BB00003010E9443230E947A0E63E580910201A3
:100BC000909103010E944E230C947A0E843879F49C
:100BD0000E944D2282FF35C067E48091020190910E
:100BE00003010E9443230E947A0E67E4E7CF9CEF43
:100BF000980F913A10F4682FE1CF90E2980F983057
:100C000050F4877091E001C0990F8A95EAF7892F17
:100C10000E94410ED9CF9BE5980F933020F480E0DD
:100C200090E00C94812298E5980F973120F480E0B1
:100C300090E00C9497228D3E20F00E9447150C9472
:100C4000BE1508951F93CF93DF93182FEB010E94D9
:100C50001005209741F08FE99FE00197F1F700C060
:100C600000002197F6CF812FDF91CF911F910C9437
:100C7000BA05893319F060E070E002C060E570E009
:100C80000C942206882321F00E943B0E0C947A0ECD
:100C90000895882321F00E94410E0C947A0E089545
:100CA000CF92DF92EF92FF920F931F93CF93DF9338
:100CB0007C01D62FC72FFC011281058102950F7090
:100CC0000E94310E8823B9F01123A9F08C2F807F68
:100CD000803421F080E28D0F883068F08091C90265
:100CE00082FD09C082E00E94DA0E0E94310E91E07E
:100CF000D82ED92601C0D12CCC2EC2948FE0C82288
:100D00008C2D90E08C30910508F0CFC1FC01EA5A9F
:100D1000FF4F0C94B32B8C2F807FCF70882311F062
:100D2000C295C07F112399F0CC2309F4AAC180E2B7
:100D30008D0F883010F0D11104C08C2F0E943B0E13
:100D400003C08C2F0E944B0E0E947A0E9AC18D2FE9
:100D50000E94BA05CC2309F4A8C180E28D0F883027
:100D600038F1DD2329F18C2F0E94510E24C08C2FE5
:100D7000807FCF70803211F0C295C07FDD2319F0E3
:100D8000D130A1F13DC08091C90282FF17C011236B
:100D900049F0CC2329F08C2F0E943B0E0E947A0E42
:100DA00080E070C180E00E94BA05CC2309F47DC1C7
:100DB0008C2F0E94410E0E947A0E77C1112371F090
:100DC000002341F0013031F40E945B0E8C2B0E9415
:100DD000630E6BC10E945B0E8C2B1DC0002319F0AB
:100DE000013009F462C10E94700E25C0112321F068
:100DF000063008F05AC10EC0053008F056C11BC0BD
:100E0000112361F0002331F0F701858180FF39C1A2
:100E10008F7085838C2F0E94420647C1002359F0B2
:100E2000D93309F03FC1FFEF07EE13E0F150004066
:100E30001040E1F735C18C2F0E94490636C18C2F36
:100E400086958695837019F0813061F02EC111234B
:100E500021F08D2F9C2F937002C080E090E00E94C3
:100E600081222BC1112321F08D2F9C2F937002C062
:100E700080E090E00E94972220C18D2F112319F06D
:100E80000E94EC1402C00E9447150E94BE1515C1B5
:100E90008C2F837009F047C011110BC12D2F2295A3
:100EA00026952770220F220F6D2F6F70862F90E0EE
:100EB000A0E0B0E0022E04C0880F991FAA1FBB1F3C
:100EC0000A94D2F7D4FF10C04FE050E060E070E029
:100ED00004C0440F551F661F771F2A95D2F740950F
:100EE00050956095709503C040E050E0BA01C695FA
:100EF000C695C3708A019B01082B192B2A2B3B2B0B
:100F0000C901B801C23049F058F4C13019F00E944B
:100F10005109CFC00E943F09CCC00E946309C9C0DB
:100F20000E943D09C6C0112319F08C2F817001C0A9
:100F30008695882309F4BDC02D2F2295269527700C
:100F4000220F220F6D2F6F70862F90E0A0E0B0E08F
:100F5000022E04C0880F991FAA1FBB1F0A94D2F744
:100F6000D4FF10C04FE050E060E070E004C0440FD8
:100F7000551F661F771F2A95D2F7409550956095AB
:100F8000709503C040E050E0BA01C695C695C370A5
:100F90008A019B01082B192B2A2B3B2BC901B80175
:100FA000C23049F058F4C13019F00E94160A81C0CD
:100FB0000E94040A7EC00E94280A7BC00E94770912
:100FC00078C0CF70112339F08C2F0E949D098D2F8E
:100FD0000E9442066EC08D2F0E9449068C2F0E94EF
:100FE000BE0967C0D23F21F128F4D03F41F0D13F84
:100FF000C1F043C0D33F19F1D43F79F03EC0112373
:1010000041F0053008F051C08C2F8F710E94E30928
:101010004CC0063008F049C0F7CF8091C90282FF6A
:1010200018C0112339F08C2F8F710E949D093DC08B
:101030001123C9F38C2F8F710E94BE0936C0112372
:1010400029F08C2F8F710E9488092FC00E9483097C
:101050002CC0112349F0CF718C2F0E949D0963E0B1
:101060008C2F0E94BF0E21C081E00E94DA0E023058
:10107000E0F082E00E94DA0E18C0112331F0002364
:1010800091F28D2F0E94100510C0002399F2D933E0
:1010900049F41FEF27EE33E0115020403040E1F7D4
:1010A00000C000008D2F0E94BA0588EF8C0D84309F
:1010B00020F40E944D220E94A504DD20C9F00E9468
:1010C0002D0E80FD15C0F70112820E94270E0E948E
:1010D0009D09C7010E9499080E94270EDF91CF91B8
:1010E0001F910F91FF90EF90DF90CF900C94BE096D
:1010F000DF91CF911F910F91FF90EF90DF90CF90F4
:1011000008950F931F93CF93DF93EC01688179814A
:101110008A810E94DF0A8C010E943A0A0E942B09F0
:10112000B801CE010E945006DF91CF911F910F911F
:101130000895CF93DF93EC01988189812B813C81C5
:10114000232B31F08F3F31F481E09F3F19F403C02E
:1011500081E001C080E080FD1DC0CE010E9423041B
:10116000811110C00E94310E8823A1F08A8188234A
:1011700089F08091C90282FD0DC082E0DF91CF919C
:101180000C94DA0ECE010E948108CE01DF91CF913E
:101190000C949E03DF91CF91089580E090E00E942F
:1011A000812280E090E00E9497220E94580E0E94C7
:1011B0007A0E0E94EF160C94BE1580910201909158
:1011C00003010E9459230C94CD080E94480E0C94F0
:1011D000DD0892959F70963079F010F4925001C01E
:1011E0009A50923068F4803F69F018F4883E40F4D9
:1011F00009C0843F29F406C0883E20F0813F11F0E9
:1012000080E0089581E00895FC01808191810E9431
:10121000D40A0E94E9080895CF93DF9300D000D04C
:101220001F92CDB7DEB70F900F900F900F900F90D9
:10123000DF91CF910895CF93DF9300D000D000D0FD
:10124000CDB7DEB726960FB6F894DEBF0FBECDBF82
:10125000DF91CF910895089508950C942C090C9472
:101260002D090E942F096093EA017093EB0180938E
:10127000EC019093ED010C94CD080C9431090F937F
:101280001F930091EA011091EB012091EC01309144
:10129000ED01602B712B822B932B1F910F910C94DE
:1012A00031090F931F930091EA011091EB012091F6
:1012B000EC013091ED0160237123822393231F9170
:1012C0000F910C9431090F931F930091EA01109133
:1012D000EB012091EC013091ED016027712782270D
:1012E00093271F910F910C9431090C942C090E94A3
:1012F00075096093E6017093E7018093E80190938C
:10130000E9010C94CD0860E070E0CB010C94770902
:101310000F931F9341E050E060E070E08A019B0171
:1013200004C0000F111F221F331F8A95D2F7C90175
:10133000B8011F910F910C9477090F931F9341E00F
:1013400050E060E070E004C0440F551F661F771F37
:101350008A95D2F78091E6019091E701A091E8018A
:10136000B091E9018A019B01082B192B2A2B3B2BF9
:10137000C901B8011F910F910C9477090F931F9326
:1013800041E050E060E070E004C0440F551F661F6C
:10139000771F8A95D2F7409550956095709580910A
:1013A000E6019091E701A091E801B091E9018A017D
:1013B0009B01082319232A233B23C901B8011F914C
:1013C0000F910C9477090F931F9341E050E060E078
:1013D00070E004C0440F551F661F771F8A95D2F72F
:1013E0008091E6019091E701A091E801B091E901B7
:1013F0008A019B01082719272A273B27C901B80121
:101400001F910F910C9477090F931F930091E601A0
:101410001091E7012091E8013091E901602B712BD7
:10142000822B932B1F910F910C9477090F931F938D
:101430000091E6011091E7012091E8013091E90166
:1014400060237123822393231F910F910C947709BA
:101450000F931F930091E6011091E7012091E8019D
:101460003091E90160277127822793271F910F91FF
:101470000C94770908952CE0929F800D1124E82F99
:10148000E695E695E695877051E001C0550F8A957F
:10149000EAF785E0E89FF0011124E853FE4F20E0D1
:1014A00030E070E04081CB01022E02C09695879516
:1014B0000A94E2F78170819584278523842781939C
:1014C0002F5F3F4F2530310569F708952CE0929F3B
:1014D000800D1124682F669566956695982F9770F4
:1014E00085E0689FB001112440E050E080E0FB01FE
:1014F000E40FF51FE853FE4F208130E0092E02C0B3
:10150000369527950A94E2F721703327042E01C0FF
:10151000220F0A94EAF7822B4F5F5F4F4530510547
:1015200031F70895BF92CF92DF92EF92FF920F931F
:101530001F93CF93DF938C01C090E601D090E70119
:10154000E090E801F090E9018091EA019091EB01CF
:10155000A091EC01B091ED01C82AD92AEA2AFB2A10
:10156000CFE1D0E0D701C6010C2E04C0B695A795F7
:10157000979587950A94D2F780FD04C0219790F73C
:10158000B12C07C0BC2EB8018C2F0E94E511019729
:10159000A9F38B2DDF91CF911F910F91FF90EF90C9
:1015A000DF90CF90BF900895CF93DF93EC010E941E
:1015B000920ABE010E94E511DF91CF9108951F9319
:1015C000CF93DF93EB019091C701992321F0CB01D9
:1015D0000E94D40A13C0882349F0CB010E94920ACA
:1015E000182F682FCE010E943B0A04C0CB010E9435
:1015F000660A182FBE01812F0E94E511DF91CF915D
:101600001F9108951F93CF93DF93C091EE0116E0D1
:101610008091EF01C81799F0D0E01C9FF0011D9F49
:10162000F00D1124E051FE4F4081518162817381A0
:10163000848195810E941B092196C770E9CFDF91B3
:10164000CF911F9108954091200250912102609105
:1016500022027091230280912402909125020C9421
:101660001B09EF92FF920F931F93CF93DF9380910B
:10167000250282958F7009F065C08091220288232F
:1016800009F460C08091EE01F090EF01109120020A
:1016900000912102609123027091240291E01F3F8A
:1016A00009F090E0C0910001D0910101292F96E04E
:1016B000E92E8F1509F446C06115710521F00F3F21
:1016C00021F030E003C031E001C0322F90E030FD66
:1016D00036C0E89EF001E99EF00D1124DF01A05113
:1016E000BE4F11963C911197301329C03C91311394
:1016F00026C012963C911297311121C013964D913C
:101700005C911497461B570B4C175D07C0F48091F2
:1017100025028F70806180932502EB50FE4F8081FF
:101720008F708061808380E292E00E949908DF914F
:10173000CF911F910F91FF90EF900C94020B0196A7
:101740008770B7CFDF91CF911F910F91FF90EF90EE
:1017500008959F92AF92BF92CF92DF92EF92FF9245
:101760000F931F93CF93DF93CDB7DEB761970FB67B
:10177000F894DEBF0FBECDBF8C0185E0F801DE011D
:101780001D9601900D928A95E1F7D8011296EC9082
:1017900090912002E09121022091230230912402B5
:1017A0002115310531F0EF3F31F481E09F3F19F40D
:1017B00003C081E001C080E0B82FB1709B2E80FD96
:1017C00047C1D8014C9111965C9111971396AD9039
:1017D000BC90149780E2C82E82E0D82EF0902202AE
:1017E000B501621B730B2091000130910101FF20B4
:1017F00009F4D9C0809125026217730708F095C0DB
:10180000282F207F09F052C05E1313C0491311C066
:10181000FE2CE1100EC08F708061809325020E9423
:10182000230BC6010E94990880912502F801858347
:101830004DC1AB2831F05F3F31F481E04F3F19F4E7
:1018400003C081E001C080E080FD03C081E08E25FF
:1018500002C080E090E0F82FF170FF2E80FF1CC0E6
:101860008091EE012091EF0136E0821709F40BC15F
:1018700090E0389FF001399FF00D1124E051FE4FA8
:101880006181561306C06081461303C06281E6126F
:1018900003C001968770E9CFFE2CEE2009F416C133
:1018A0008091250281608093250254C05E1306C09A
:1018B000491304C0E11002C0F80199C0C8010E9498
:1018C0000409882361F1EE2051F120912502822F35
:1018D00082958F7090E0029774F080912002909131
:1018E000210298878F831986BB86AA862C87CE0112
:1018F00007960E94990886E0F801A0E2B2E0019004
:101900000D928A95E1F70E94310B0E94230B0AC0C9
:101910005E1711F1C8010E94040981112CC0C80191
:101920000E949908FF24F394D1C0282F207F81F7CB
:101930007A2DB98AA88A6E2D89890E940C0980E2C5
:1019400092E00E94990886E0D6011D928A95E9F7F7
:101950000E94230BF12CBAC04913DCCFE110DACF7F
:10196000F8018583C8010E94990886E0D6011D927E
:101970008A95E9F7ABC0EE2091F220912502822FE3
:1019800082958F7090E002970CF4B5CF8091200281
:10199000909121029A8389831B82BD82AC822E831F
:1019A000CE010196A6CF6217730708F044C0FE2C43
:1019B000EE2009F4B4CF5E1330C049132EC020913D
:1019C000250220FD21C0822F82958F70482F50E084
:1019D00041155105C9F0F80125834F30510541F0FB
:1019E0008F5F982F9295907F822F8F70892B8583A0
:1019F000C8010E94990886E0F801A0E2B2E00190D7
:101A00000D928A95E1F73CC086E0F801A0E2B2E0D1
:101A100001900D928A95E1F759C0C8010E9404090E
:101A2000811169CF80912502816080932502C801D0
:101A30000E9499084BC07A2DB98AA88A6E2D89898F
:101A40000E940C0986E0D6011D928A95E9F718C01C
:101A5000EE2009F464CFC8010E940409F82E8823FF
:101A600009F45DCF86E0F801A0E2B2E001900D92AA
:101A70008A95E1F780E292E00E940A050E94310B0C
:101A80000E94230B23C04D875E878D859E850E9413
:101A9000D40A292F22952F70223028F49F7039F014
:101AA000811105C00BC0243028F49F7049F4805E7A
:101AB000883020F0C8010E9499089F2CF92C06C09C
:101AC000D80115969C91907F91F7F8CF8F2D619654
:101AD0000FB6F894DEBF0FBECDBFDF91CF911F913F
:101AE0000F91FF90EF90DF90CF90BF90AF909F90BD
:101AF00008951F93CF93DF93CDB7DEB72C970FB622
:101B0000F894DEBF0FBECDBF4F83588769877A87B1
:101B10008B879C87CE0107960E94A90B8823D1F062
:101B20009F8188852A853B85232B31F08F3F31F4B7
:101B300081E09F3F19F403C081E001C080E080FD97
:101B400047C04F81588569857A858B859C850E9421
:101B50001B093EC086E0FE013796DE01119601901A
:101B60000D928A95E1F7FF81E8856A857B8561158D
:101B7000710531F0EF3F31F481E0FF3F19F403C00C
:101B800081E001C080E080FD23C02091EF0130E0C2
:101B9000C9010196877099274091EE0150E08417A2
:101BA0009507F1F1F983EA837D836C8396E0929F38
:101BB000D001939FB00D1124A051BE4FFE0131966C
:101BC00001900D929A95E1F78093EF010E94020B2C
:101BD00016E08091EE019091EF01891771F1189F45
:101BE000C001112480519E4F0E94A90B882329F126
:101BF000E091EE011E9FF0011124E051FE4F408163
:101C0000518162817381848195810E941B09809139
:101C1000EE0190E00196877099278093EE01D9CF6D
:101C20000E94E5081092EF011092EE01E0E2F2E06E
:101C300086E0DF011D928A95E9F72C960FB6F8949D
:101C4000DEBF0FBECDBFDF91CF911F910895809170
:101C50004602859585958595089580914602877001
:101C6000089590914602977081E009F480E008950C
:101C700080916902089590916902892B809369028D
:101C8000089580959091690289238093690208954F
:101C900010926902089590916802892B80936802DE
:101CA0000895809590916802892380936802089531
:101CB00010926802089580914702089508950C9447
:101CC0005E0E0C945F0E9091C90292FD08C0909137
:101CD0004702981721F0809347020C94610E0895F3
:101CE00080914702882329F01092470280E00C94EB
:101CF000610E0895CF93DF93E0910201F09103010B
:101D0000809169028083E0910201F091030190814A
:101D100080916802892B808380914702882381F01B
:101D2000E0910201F09103019081892B80838091E1
:101D30000201909103010E94AD2281110E94700E58
:101D4000C0910201D091030140E250E066E272E0EE
:101D5000CE010E94F72B892B69F080E2FE01A6E2FA
:101D6000B2E001900D928A95E1F7CE01DF91CF911B
:101D70000C945922DF91CF9108950C945E0E9091AE
:101D8000C90292FD10C098E0899F90011124262B72
:101D9000209346020E949D09809146028595859573
:101DA00085950C94BD0E0C949D091092460280E01E
:101DB0000C94BD0E209146028095822380934602AA
:101DC000982F977099F430E0482F082E000C550B8F
:101DD0002417350759F09091C90292FD07C08595E7
:101DE000859585950E94BE090C94D50E0895909115
:101DF000C90292FB222720F9281769F080FB92F98B
:101E00009093C9028091C8029091C9020E94450F27
:101E100082E00C94DA0E08958091C90282FB882733
:101E200080F991E089270C94F70E81E00C94F70E6D
:101E300080E00C94F70E6FEF7FEF80E090E00C9461
:101E4000362C80E090E00E94122C21E0893E9E4FCB
:101E500009F020E0822F089582E090E00C94042C99
:101E600083E090E00C94042CCF9384E090E00E94F7
:101E7000042CC82F82E290E00E94042C2C2F30E02A
:101E8000A901582BCA01CF910895CF93C92F682F6C
:101E900084E090E00E94182C6C2F82E290E0CF91B9
:101EA0000C94182CAB01BC018FE090E00C942A2C10
:101EB000AB01BC0183E190E00C942A2C60E070E05F
:101EC000CB010C94580F60E070E0CB010E94520FE0
:101ED0000C945E0F69EE7EEF80E090E00E94362C5D
:101EE00060E082E090E00E94182C60E083E090E0E7
:101EF0000E94182C1092EA011092EB011092EC0152
:101F00001092ED0160E084E090E00E94182C60E007
:101F100082E290E00E94182C60E085E090E00E9450
:101F2000182C60E086E090E00E94182C6FEF87E0AC
:101F300090E00E94182C40E050E0BA0188E090E068
:101F40000E942A2C60E08DE090E00E94182C40E076
:101F500050E0BA0188E190E00E942A2C60E087E11D
:101F600090E00E94182C40E050E0BA018CE190E033
:101F70000E942A2C60E070E080E290E00E94362C03
:101F800040E050E0BA0188E190E00E942A2C0C94D5
:101F9000630F0C946A0F682F8EE090E00C94182C5D
:101FA0000E941324609376027093770280937802E4
:101FB000909379026093720270937302809374021B
:101FC00090937502089585B7806885BF85B780684E
:101FD00085BF089581E008950C94EA0F08950C944C
:101FE000EE0F0C94EE0F0C94F10F0C94EE0F0C947A
:101FF000F50F0C94EE0F0E94E30F81EC92E10E942A
:1020000043220E94F90F0C94F70F0E94EF0F0C94DB
:10201000EE0F0E94DB120E94A2040C94CA1F0E94C1
:10202000FE230E94C0130E9409100E94081E0E94F5
:10203000471C0C94F30F5F926F927F928F929F9246
:10204000AF92BF92CF92DF92EF92FF920F931F93C6
:10205000CF93DF93CDB7DEB72A970FB6F894DEBFE4
:102060000FBECDBF0E94D513C82E81110E94D00F84
:102070003AE6832E32E0932E00E010E0502E802FBF
:102080000E94FF125C01F401619071904F0168267B
:10209000792661147104B1F40F5F1F4F04301105EC
:1020A00069F78FEF89838A831B820E9407248160EE
:1020B000782F9D838C8349815A816B818D810E9409
:1020C000C0043AC080917A0281FD0E940813D12C8D
:1020D000EE24E394F12CC3018E219F21892B29F159
:1020E0000E94EC0F8823A9F0DE825F82AE20BF2021
:1020F00081E0AB2809F480E088870E940724816092
:10210000782F9A8789874E815F8168858A850E94AA
:10211000C004000F111FF801E659FD4F8081918125
:10212000E826F926F182E08207C0D394EE0CFF1C6A
:10213000FCE0DF12D0CFB0CF81E0C11001C080E061
:102140002A960FB6F894DEBF0FBECDBFDF91CF91B8
:102150001F910F91FF90EF90DF90CF90BF90AF90C5
:102160009F908F907F906F905F9008950E941B10BA
:102170000E947A1C0E94C91F0E94DC150C94B504B1
:10218000CF93DF930E94EA11EC01811521E59207BC
:1021900008F045C0811530E5930708F094C0883EEB
:1021A000910528F5803E910508F0F8C0883A910520
:1021B00070F4853A910508F07CC08130910509F4EE
:1021C00075C008F4E8C0049708F0E8C0E4C08F3B8D
:1021D000910508F0E0C0C85AD0E0CC0FDD1FC35A0B
:1021E000DE4F0990D881C02DCE019464D8C08115EE
:1021F00040E2940758F4811551E0950708F0CEC0ED
:102200008D3E910508F4C7C09065C9C0C11580E432
:10221000D80708F4C0C0DF70CE01906AC0C0811535
:1022200025E59207A8F4811534E5930708F095C0D9
:10223000811543E5940708F07BC0811552E59507A9
:1022400008F061C0D82FCC27CE01816F906AA7C05B
:10225000C11589E5D807A0F4C11528E5D20708F013
:1022600082C0C11536E5D30708F095C08C2F0E94B7
:102270007E128F7190E0D82FCC27CE0190628FC054
:10228000C1154AE5D40708F474C0CE0190568115F3
:10229000904208F080C08D2F8F710E947E12DD2742
:1022A000D0628F71AE01582BCA0179C081E090E0F5
:1022B00076C0C55AD0E0C557DE4F8881C82FD0E020
:1022C000CE0190646CC074E0969587957A95E1F79D
:1022D000282F23703C2F337081E090E002C0880FDC
:1022E000991F3A95E2F79C68AC01522B9A019C2FFA
:1022F0009F709695969550E2959FE0011124C90133
:102300008C2B9D2B4CC08370992721E030E002C0BC
:10231000220F331F8A95E2F79C2F9695969580E2BF
:10232000989FE0011124C22BD32BCE019C6837C0AB
:102330008370992721E030E002C0220F331F8A9575
:10234000E2F79C2F9695969540E2949FE001112428
:10235000C22BD32BCE019A6822C0D82FCC27CE0116
:10236000846F906A1CC0DC2FCC27CE01806F906AEE
:1023700016C08C2F8F700E947E1294E0D695C79560
:102380009A95E1F7CF70D0E0DC2FCC27D0699E0181
:10239000282BC90104C080E090E001C0CE01DF918C
:1023A000CF91089520E3829FC0011124FC012CE00D
:1023B000729FE00DF11D1124E60FF11DEE0FFF1FBE
:1023C000E852FF4F8591949108950E94D2110E9486
:1023D000C01008958238910569F1B0F481339105F8
:1023E00009F46DC048F48932910509F463C08A325A
:1023F000910509F469C008958533910509F455C024
:1024000089339105B9F00895833E910569F138F457
:10241000803E9105B1F0823E910509F10895863E16
:102420009105A9F1873E9105B9F1843E910509F026
:1024300064C023C02091C80220FD4FC021FD4DC0C3
:1024400008958091C80280FD44C08091C90280FF38
:1024500044C08091C80284FD42C083EE4DC080918B
:10246000C80282FF38C0F5CF8091C80282FD33C018
:102470008091C90280FD31C0ECCF8091C90281FFFB
:1024800032C08091C80284FD2AC087EE35C0809199
:10249000C80283FF26C0F5CF8091C80283FD21C00A
:1024A0008091C90281FD1FC0ECCF8091C80285FDDB
:1024B0001CC01DC08091C80285FD19C016C0809146
:1024C000C80286FD16C017C08091C80286FD13C0E1
:1024D00010C089E311C082EE0FC080EE0DC080E015
:1024E0000BC086EE09C084EE07C089E205C085E313
:1024F00003C08AE201C081E390E008959091C80290
:1025000092FF0DC0282F2871283019F4877F84602E
:1025100006C0282F2471243011F48B7F886093FF2C
:102520000DC0282F2871283119F4877E846106C0D8
:10253000282F2471243111F48B7E88612091C902E7
:1025400020FF0DC0382F3871383019F4877F816033
:1025500006C0382F3171313011F48E7F886021FF31
:102560000DC0282F2871283119F4877E816106C09B
:10257000282F2171213111F48E7E886194FD877E90
:10258000089580E008950C941B0F0E94D5138FE3EB
:102590009CE90197F1F700C000000E94D51380E08C
:1025A0000E94FF1280FF04C00E94C3120C945424A6
:1025B00008950C94C5120E94210F811102C00E943F
:1025C000C90F0E942C0F80937A020E94340F9093BF
:1025D000C9028093C8020E94D9120E94300F682F4E
:1025E00070E080E090E00E943D096091E60170910A
:1025F000E7018091E8019091E9010C947509E82FB9
:10260000F0E0EE0FFF1FEE52FD4F808191810895A3
:10261000089580EA8A95F1F7089500C008950C9412
:10262000091308950C9411130C9412130C941113A4
:102630000C941613F894E82FE295EF70F0E031A1B6
:10264000282F2F7081E090E001C0880F2A95EAF7CB
:10265000982F9095932391A392A1892B82A378948C
:1026600008950F931F93CF93DF93CAE9D1E0899127
:102670008F3F11F00E941A1381E0CE39D807B9F7C5
:10268000CEE8D1E00AE911E089918F3F11F00E9474
:102690001A130C171D07C1F7DF91CF911F910F91EE
:1026A0000895BF92CF92DF92EF92FF920F931F9304
:1026B000CF93DF938C01C62FD0E0CE0186569E4F7C
:1026C0006C01FC0190819F3F09F450C0B62EF89434
:1026D000E92FE295EF70F0E081A19F7021E030E0FA
:1026E00001C0220F9A95EAF7822B81A382A120953F
:1026F000282322A378940E940D13EEE8F1E04AE922
:1027000051E021E030E0E12CF12C61916F3F89F044
:10271000A62FA295AF70B0E090968C9190E06F706C
:1027200002C0959587956A95E2F780FD02C0C901C0
:1027300002C080E090E0E82AF92A220F331F4E17EA
:102740005F0719F7F60180818F3F11F00E941A137D
:1027500061E0E114F10409F460E08B2D0E940F1395
:10276000CC0FDD1FC00FD11FF982E882DF91CF911E
:102770001F910F91FF90EF90DF90CF90BF90089541
:102780000E94311388E0E2EDF2E0DF01982F1D9204
:102790009A95E9F7EAECF2E0DF011D928A95E9F7F4
:1027A00084E00E9420140C940F04FF920F931F9357
:1027B000CF93DF93CDB7DEB728970FB6F894DEBF7F
:1027C0000FBECDBF8E010F5F1F4F88E0F801119241
:1027D0008A95E9F7F12C6F2DC8010E945113F394EB
:1027E000F4E0FF12F8CF48E050E0B8018AEC92E044
:1027F0000E94F72BFF24F394009709F4F12C892B06
:1028000041F088E0F801AAECB2E001900D928A95BF
:10281000E1F72F2D44E062ED72E08AEC92E00E9435
:1028200021140E9411048F2D28960FB6F894DEBF54
:102830000FBECDBFDF91CF911F910F91FF900895F3
:102840000895FF920F931F93CF93DF93F82E092FD4
:10285000162FD72FC42F222349F081E080937D02C9
:102860000E94072490937C0280937B0280917D02DA
:102870008823D9F080917B0290917C020E941F24D2
:10288000059798F0EF2DF02FA12FBD2F80E090E05D
:102890004C2F50E08417950734F4219131912D93FA
:1028A0003D930196F7CF10927D02DF91CF911F915A
:1028B0000F91FF9008950E941F260E940F100C9404
:1028C0002B260E942F260E94B6100C9449260E94A7
:1028D000A5230E9406260E94FB0F0E945B140E9403
:1028E00061140E940510FBCF8091840280FF06C016
:1028F0006091090170E0660F771F26C081FF04C058
:102900006091090184E005C082FF07C06091090160
:1029100088E0689FB001112417C090918302992329
:10292000D1F060910801961788F72091090188E09D
:10293000289F90011124929FA001939F500D112474
:1029400070E0CA010E947D2B6038710540F461156A
:10295000710519F406C068E070E0862F08958FE7CE
:10296000089581E008958091840280FF08C06091FD
:10297000050170E0759567957595679521C081FF94
:1029800006C06091050170E07595679519C082FFDA
:1029900004C06091050170E010C0909182029923FB
:1029A00099F0609104019617A0F780910501899F25
:1029B000C001112470E00E947D2B6038710540F445
:1029C0006115710519F406C061E070E0862F089565
:1029D0008FE7089581E008958D3E21F40E947414DC
:1029E000819504C08E3E29F40E947414809388025D
:1029F00008958F3E21F40E947414819504C0803F95
:102A000029F40E947414809387020895893F19F471
:102A10000E94B31405C08A3F31F40E94B31481951B
:102A20008093890208958B3F21F40E94B31481950D
:102A300004C08C3F29F40E94B31480938A02089545
:102A40009FE0980F983078F421E030E0A90102C0AF
:102A5000440F551F9A95E2F7CA0190918602892B7F
:102A60008093860208958D3F21F4809184028160D5
:102A70000BC08E3F21F480918402826005C08F3F9D
:102A800029F48091840284608093840208958D3EAD
:102A900039F49091880297FF35C01092880259C08E
:102AA0008E3E29F4909188021916BCF32BC09091A8
:102AB00087028F3E29F497FF25C01092870249C0F4
:102AC000803F19F41916CCF31DC090918902893FFB
:102AD00029F41916BCF4109289023BC08A3F19F4FC
:102AE00097FF10C0F8CF8B3F39F490918A0297FF7F
:102AF00009C010928A022DC08C3F21F490918A0265
:102B00001916BCF39FE0980F983080F421E030E074
:102B1000A90102C0440F551F9A95E2F7CA0180959A
:102B20009091860289238093860213C08D3F21F401
:102B3000809184028E7F0BC08E3F21F480918402AD
:102B40008D7F05C08F3F29F4809184028B7F809315
:102B5000840280918702811106C0809188028111D0
:102B600002C01092830280918902811106C0809177
:102B70008A02811102C01092820208950E940724E5
:102B800020918702211104C020918802222321F084
:102B9000909381028093800220918902211104C0C8
:102BA00020918A02222321F090937F0280937E025B
:102BB00085E892E00C947322EF92FF920F931F939B
:102BC000CF93DF9300D000D000D0CDB7DEB786E042
:102BD000E5E8F2E0DE01119601900D928A95E1F7A9
:102BE000E0908702F09088020091890210918A0299
:102BF00010928702109288021092890210928A0223
:102C0000E11003C0FF2009F45DC080918002909123
:102C100081020E941F24AC0190918302992339F014
:102C200020910A0130E02417350758F04BC020915D
:102C30000B018AE0289F900111242417350718F012
:102C400041C09F3F19F09F5F90938302EE2061F097
:102C50000E9474141E1414F09FEF01C091E0989F1D
:102C6000902D112490938702FF2061F00E9474142C
:102C70001F1414F09FEF01C091E0989F902D112434
:102C800090938802309187023323E1F020918802EB
:102C90002223C1F045EB3403C0011124992319F01C
:102CA0009093870203C081E08093870235EB230372
:102CB000C0011124992319F09093880203C081E088
:102CC00080938802011103C0112309F45DC0809133
:102CD0007E0290917F020E941F24AC01909182029B
:102CE000992339F02091060130E02417350758F078
:102CF0004BC0209107018AE0289F900111242417DE
:102D0000350718F041C09F3F19F09F5F90938202F2
:102D1000002361F00E94B314101614F09FEF01C05D
:102D200091E0989F902D112490938902112361F0D6
:102D30000E94B314111614F09FEF01C091E0989F08
:102D4000902D112490938A02309189023323E1F06F
:102D500020918A022223C1F045EB3403C0011124E3
:102D6000992319F09093890203C081E0809389022E
:102D700035EB2303C0011124992319F090938A02A3
:102D800003C081E080938A028091870281110BC089
:102D900080918802811107C080918902811103C04E
:102DA00080918A0281110E94BE15EB82FC820D8304
:102DB0001E8386E0FE013196A5E8B2E001900D92F7
:102DC0008A95E1F726960FB6F894DEBF0FBECDBF09
:102DD000DF91CF911F910F91FF90EF900895E5E85B
:102DE000F2E086E0DF011D928A95E9F710928302F6
:102DF00010928202109284020895EF92FF920F9334
:102E00001F93CF93DF938B01682F11110AC04423C6
:102E100029F0E82FF0E0E159FC4F6491762F862FDE
:102E200075C0212F30E0E82FF0E0442321F0E15974
:102E3000FC4FE491F0E046E0049FC0011124CFEF85
:102E4000D0E0BE010E94692B4BEA4603C001479FB8
:102E5000900D1124800F911D800F911D982F990FB7
:102E6000890FAE01421B530B4E9FD0014F9FB00DF7
:102E70005E9FB00D11249B2F189FA0011124452F98
:102E800055278E01041B150B0E9FA0010F9F500D9F
:102E90001E9F500D11247E01E81AF108E29E800168
:102EA000E39E100DF29E100D1124212F3327C21B1B
:102EB000D30BCE9F9001CF9F300DDE9F300D11249C
:102EC00062307105A9F048F46115710569F061304F
:102ED0007105C9F48B2F752F0DC06430710581F019
:102EE00058F06630710579F47E2F8B2F932F0DC02B
:102EF000832F7B2F9E2F09C08E2F7B2F952F05C0F0
:102F00008E2F732F02C07E2F852F692FDF91CF91D7
:102F10001F910F91FF90EF90089541E00E94FD16E0
:102F2000089508950E948D170895CF93DF93762F0B
:102F3000E901682F842F0E949217798368838A831E
:102F4000DF91CF9108958091DA02282F269530E005
:102F50002115310519F48170826005C025323105D3
:102F600024F0817088648093DA02089588E090E00C
:102F70000C940C2CCF92DF92EF92FF926B017C01AC
:102F80000E94A317B701A60188E090E0FF90EF90A0
:102F9000DF90CF900C942A2CEAEDF2E083E080835E
:102FA00011828FEF82838383148260817181828199
:102FB00093810C94BA178091DA0280FF02C0869543
:102FC000089580E008959091DE02933018F49F5F99
:102FD0009093DE02882351F06091DA027091DB0257
:102FE0008091DC029091DD020C94BA17089581E083
:102FF0000C94E3179091DE02992319F0915090936D
:10300000DE02882351F06091DA027091DB02809138
:10301000DC029091DD020C94BA17089581E00C94C3
:10302000FA1770E00C94DA1F609110018091DA02B7
:1030300080FF0AC080910F0123E0829FC00111240C
:1030400081529D4F0C9411188091110190911201A1
:10305000891780F7E82FF0E09F01220F331FE20F5E
:10306000F31FE152FD4F1182108212828F5FF0CF69
:103070009091DA0290FF16C09091110120911201F7
:10308000921770F4E92FF0E0DF01AA0FBB1FEA0FDF
:10309000FB1FE152FD4F8183608342839F5FF0CF2E
:1030A0000C9414180895CF93DF9300D01F92CDB7DE
:1030B000DEB79091DA0290FF0AC09E012F5F3F4F6A
:1030C0000E9495174B8169818A810E9438180F9060
:1030D0000F900F90DF91CF910895CF93DF93EC0184
:1030E000EC81F0E0E659FD4F4491EAEDF2E06281B7
:1030F00081810E9453188C818F5F8C83DF91CF91E7
:103100000895CF93DF93EC01EAEDF2E04381628111
:103110008C810E9453188C818F5F8C83DF91CF91BB
:1031200008950F931F93CF93DF9300D01F92CDB7D5
:10313000DEB78C0180918B0281110AC09E012F5F46
:103140003F4F4FEF6FEF0E9495178A8180938B025C
:10315000F8018481813051F028F0823061F440918F
:103160008B020AC080918B0240E007C060918B0205
:1031700040E080E003C040E080E060E00E9438185A
:10318000F801848190E0019663E070E00E947D2B5D
:1031900084830F900F900F90DF91CF911F910F912B
:1031A0000895AF92BF92CF92DF92EF92FF920F936A
:1031B0001F93CF93DF9300D01F92CDB7DEB7182FA8
:1031C000F62E042FE22E9091DA0290FF6DC0E92FC7
:1031D000E695AE2FB0E0A256BE4F8C91809395023B
:1031E0009E7F923061F49E012F5F3F4F812F0E949E
:1031F00095174B8169818A810E94381843C08230BB
:1032000019F40091DD023EC0863019F41091DB0202
:1032100039C08930D9F38931A9F5E9518E2F8170F0
:10322000D82EE695F0E0E659FC4FA590B490C12C5D
:10323000BB2460911301C61618F52C2D30E0A29E18
:10324000C001A39E900DB29E900D112470E00E94CB
:10325000692B812FD11002C0860F01C0861B90916F
:103260001101290F311DA901440F551F240F351FCE
:1032700021523D4F402F6F2D0E949517C394D9CFF7
:103280000E9414181093DB02F092DC020093DD021E
:10329000EE2051F06091DA027091DB028091DC0245
:1032A0009091DD020E94BA170F900F900F90DF915E
:1032B000CF911F910F91FF90EF90DF90CF90BF9033
:1032C000AF900895EAEDF2E09181282F4381628169
:1032D0008AE0890F0C94D11881E00C946219EAED10
:1032E000F2E09181282F4381628186EF890F0C944F
:1032F000D11881E00C946F19EAEDF2E0628121E1CE
:10330000620F08F46FEF282F438181810C94D1184C
:1033100081E00C947C19EAEDF2E0628121E1621B0C
:1033200008F460E0282F438181810C94D11881E05A
:103330000C948B19EAEDF2E0438121E1420F08F48D
:103340004FEF282F628181810C94D11881E00C9479
:103350009A19EAEDF2E0438121E1421B08F440E0D2
:10336000282F628181810C94D11881E00C94A919D5
:1033700020E00C94D118FF920F931F93CF93DF930B
:10338000EC01F12C0FEF10E060911301F616F0F450
:10339000809111012F2D30E0280F311DC901880FB8
:1033A000991F280F391F21523D4F70E0C8010E941C
:1033B0007D2B962F8C814091DD026091DC02F99E7D
:1033C000800D11240E949517F394DECF0E941418EB
:1033D0009A818C8190FF02C08F5F01C081508C83E5
:1033E000DF91CF911F910F91FF900895BF92CF92DF
:1033F000DF92EF92FF920F931F93CF93DF93FC0125
:10340000828180FF02C00FEF01C001E010E08091D7
:103410001301181708F040C080911101C12ED12C62
:10342000E601C80FD11DCE01880F991FC80FD91F03
:10343000C152DD4F198218821A8234E0E32EF12C3A
:10344000B12C80918D028B0D853014F0837005C0F6
:1034500087FF03C090911301890F082E000C990B70
:10346000C816D90691F48091DD028E9DA0018F9D32
:10347000500D112455954795559547959E0160919E
:10348000DC028091DB020E949517B00EF1E0EF1A8A
:10349000F108B9F61F5FBBCF0E94141880918D020E
:1034A000013031F4811102C080911301815007C0B5
:1034B00090E001966091130170E00E947D2B809353
:1034C0008D02DF91CF911F910F91FF90EF90DF90D0
:1034D000CF90BF900895CF938091110190911201E8
:1034E000891770F4E82FF0E09F01220F331FE20FDD
:1034F000F31FE152FD4F1182108212828F5FF0CFD5
:10350000C0E060911301C617C0F5EC2FF0E070E049
:10351000CF010E947D2B20911101820F20918C02FE
:10352000022E000C330B90E0E217F307CCF0209151
:103530000E01022E000C330B2E173F078CF09C015E
:10354000220F331F820F931F9C0121523D4F409148
:10355000DD026091DC028091DB020E9495170BC0B6
:10356000FC01EE0FFF1F8E0F9F1FFC01E152FD4F6C
:10357000118210821282CF5FC4CF0E941418209152
:103580000D0180918C02820F80938C0290910E012C
:10359000920F90930E0119165CF4082E000C990BF3
:1035A0004091130150E041505109841795071CF0D8
:1035B000219520930D01CF9108958F929F92AF9204
:1035C000BF92CF92DF92EF92FF920F931F93CF9310
:1035D000DF938C01FC014481C42FD0E09E01DE0109
:1035E0000E94C12B9B01AC010E94D72B6B017C0177
:1035F000E0E2F0E0EC1BFD0BA5E5B0E09B01AC01C7
:103600000E94D72B4B015C019F01DF010E94B92B67
:103610009B01AC010E94E22B9B01AC012C0D3D1DD6
:103620004E1D5F1DC501B4010E94912BC22FD22FE8
:103630002A3228F4F3E02F9F900111240DC025E5D4
:1036400030E02C1B3109C901880F991F280F391F41
:1036500037FF02C02F5F3F4F35952795C22FC0958A
:10366000F12C85E5E82EED1A80911301F816C8F4C7
:10367000F1FC02C08E2D01C08D2F909111012F2DD4
:1036800030E0290F311DA901440F551F240F351FAC
:1036900021523D4F4C2F6091DC020E949517F3940C
:1036A000E3CF0E941418F8018481811102C091E0D7
:1036B00003C0803219F49FEF90930C0190910C019C
:1036C000890FF8018483DF91CF911F910F91FF90B3
:1036D000EF90DF90CF90BF90AF909F908F90089524
:1036E0000F931F93CF93DF93EC0100E010E08091E4
:1036F0001301282F30E00217130724F590911101D0
:103700009801290F311DA901440F551F240F351FA2
:1037100021523D4F869590E04C81081719071CF403
:10372000442331F002C0411103C04091DD0201C0C9
:1037300040E06091DC028091DB020E9495170F5FF0
:103740001F4FD5CF0E9414188C8190E00196817094
:1037500099278C83DF91CF911F910F910895EAED06
:10376000F2E080818E7F808360817181828193818C
:103770000E94BA17109296022FEF80E792E0215034
:1037800080409040E1F700C000000C941418609154
:10379000DA02669570E04BE050E084E191E00E942F
:1037A000EA2B892B19F481E0809396020E9407246A
:1037B00090938F0280938E0208959091DA0290FF89
:1037C00035C09170811102C0926006C0853210F040
:1037D000986402C0880F982B9093DA02662351F008
:1037E0006091DA027091DB028091DC029091DD023F
:1037F0000E94BA176091DA02669570E04BE050E0E3
:1038000084E191E00E94EA2B892B19F01092960234
:1038100002C00E94C71B81E0809391024091DD02AB
:103820006091DC028091DB020C94B8190895682F36
:103830009091DA02969581E0890F853208F081E057
:103840000C94DD1B81E00C94171C682F9091DA0218
:1038500096958FEF890F09F484E20C94DD1B81E0CB
:103860000C94251C61E00C94DD1BEAEDF2E08081F4
:103870008160808386950C94321C8091DA0280FDF1
:103880000C94AF1B0C94351C60E00C94DD1B8091F4
:10389000940281112EC00E94210F811104C00E9448
:1038A000C90F0E94CC170E94B6176093DA0270937A
:1038B000DB028093DC029093DD026E7F61F40E9454
:1038C000CC170E94B6176093DA027093DB028093E4
:1038D000DC029093DD020E94A31710929602809161
:1038E000DA0280FF03C086950E94441C81E0809329
:1038F000940208950F931F93CF93DF9380919602C4
:10390000882309F485C080919502E091DA02E6955A
:10391000E81BE0939002823049F4F0E0EA59FD4F51
:10392000E491CE2FD0E00DE618E149C0863049F48D
:10393000F0E0ED59FD4FE491CE2FD0E001E818E121
:103940003EC0893051F4E695F0E0E05AFD4FE49135
:10395000CE2FD0E00BEB19E132C08F3051F4E69559
:10396000F0E0E35AFD4FE491CE2FD0E006EF19E1ED
:1039700026C0853149F4F0E0E65AFD4FE491CE2FA0
:10398000D0E00BE61AE11BC0883181F0833239F4B4
:10399000E8E5F2E0C591D49101E918E110C0843264
:1039A00051F4C4EFD1E000E71BE109C0C8E2D0E068
:1039B0000DED1AE104C0C0EDD7E001E917E18091F7
:1039C0009102882361F0109291020E940724909343
:1039D0008F0280938E0210929302109292020E94A4
:1039E0000724E0918E02F0918F028E1B9F0B8F3F78
:1039F0009F4770F4EC0FFD1FF0938F02E0938E024F
:103A00008EE892E0F801DF91CF911F910F91099418
:103A1000DF91CF911F910F910895882311F0FA0142
:103A200001C0FB010994CF93DF93C82FD62F0E94CA
:103A3000DB178C1740F00E94DB178D1720F4DF9105
:103A4000CF910C94221C8C2FDF91CF910C94321CBF
:103A50001F93CF93DF93FB0112811111C3C0EC01BF
:103A60000E94380E8272CD3CFCE5DF0709F49AC053
:103A7000A8F5C73CECE5DE0709F476C0A8F4C43C21
:103A80009CE5D90709F45FC028F4C33CDC4509F480
:103A900057C054C0C53C9CE5D90709F459C0C63C81
:103AA000DC4509F45CC04AC0CA3CFCE5DF0709F408
:103AB0006AC050F4C83CECE5DE0709F45AC0C93CC2
:103AC000DC4509F45BC03AC0CB3C9CE5D90709F45E
:103AD0005FC0CC3CDC4509F460C030C0C23DFCE5B1
:103AE000DF0709F46FC088F4CF3C9CE5D90709F4DF
:103AF00060C008F45CC0C03DFCE5DF0709F45CC0B1
:103B0000C13DDC4509F45BC019C0C53D9CE5D90742
:103B100009F460C050F4C33DFCE5DF0709F455C06B
:103B2000C43DDC4509F454C009C0C63D9CE5D90735
:103B300009F455C0CE35DD4509F454C011E052C03A
:103B40000E943D1C4FC04FE25CE162E27CE104C098
:103B500042E25CE16FE27CE10E940D1D43C049E757
:103B600059E16CE679E1F8CF4CE659E169E779E192
:103B7000F3CF47E959E168E879E1EECF48E859E148
:103B800067E979E1E9CF45EB59E166EA79E1E4CF0C
:103B900046EA59E165EB79E1DFCF4EE058E167EFA6
:103BA00077E1DACF47EF57E16EE078E1D5CF81E0FA
:103BB00017C065E082E010C068E086E00DC06EE0EE
:103BC00089E00AC064E18FE007C067E185E104C0D5
:103BD00088E106C062E289E10E94131D03C083E20E
:103BE0000E94321C812FDF91CF911F91089586E0B2
:103BF00090E00C94042C682F86E090E00C94182C34
:103C00008091EB02847081628093EB020C94FB1D27
:103C10000E94210F811104C00E94C90F0E94001E42
:103C20000E94F71D8093EB02282F26952695269556
:103C300030E02530310524F0877080628093EB02FC
:103C40008091EB0280FF04C086958695869501C021
:103C500080E00C94191F2091EB02822F86958695A7
:103C60008695482F50E04430510554F48F5F982FCB
:103C7000990F990F990F822F8770892B8093EB02F0
:103C80008091EB0281608093EB020E94FB1D80918A
:103C9000EB028695869586950C94191F8091EB0210
:103CA000982F969596959695A1F0915E990F990FFC
:103CB000990F8770892B8093EB02887F91E009F43C
:103CC00090E08091EB0290FB80F98093EB020E94E0
:103CD000FB1D8091EB028695869586950C94191FA5
:103CE0008091EB0280FD13C081608093EB028130F4
:103CF00019F489E08093EB028091EB020E94FB1D96
:103D00008091EB028695869586950C94191F0895EF
:103D10008091EB0280FF08C08E7F8093EB020E94AF
:103D2000FB1D80E00C94191F08958091EB0280FD2B
:103D30000C94881E0C94701E9091EB02892F86952E
:103D4000869586958F5F8F719770853038F4880FD0
:103D5000880F880F892B8093EB0202C09093EB02AF
:103D60008091EB02887F91E009F490E08091EB0272
:103D700090FB80F98093EB020E94FB1D8091EB0287
:103D80008695869586950C94191F853008F084E0F9
:103D90009091EB029770282F220F220F220F922B67
:103DA0009093EB02987F21E009F420E09091EB02E0
:103DB00020FB90F99093EB020C94191F0E94C51EF2
:103DC0008091EB020C94FB1D9C01FB0182818823F6
:103DD00049F12E3BFCE53F07C9F040F42C3BECE5F4
:103DE0003E0769F02D3B3C4561F00895203C9CE581
:103DF000390791F070F0213C3C4589F0089584E04A
:103E000001C080E00E94DE1E80E008950E944E1EE8
:103E1000FBCF0E942B1EF8CF0E94951EF5CF0E946B
:103E20009C1EF2CF81E00895269A2E9808952E9830
:103E300008958F929F92AF92BF92CF92DF92EF92AE
:103E4000FF920F931F93CF93DF93C82F853050F4C9
:103E5000811109C0809180008F7D809380000E9435
:103E6000171F06C0C4E080918000806280938000AC
:103E7000A0918600B09187002C2F30E00E94C12BCA
:103E80008B019C0142E036952795179507954A9539
:103E9000D1F780918600909187006CE070E00E94DD
:103EA000692B6017710730F0C80169E070E00E946B
:103EB000692B5EC08091860090918700E09086001B
:103EC000F0908700E0918600F0918700C6E0D0E096
:103ED000BE010E94692B060F171F211D311D4801CD
:103EE000590185E0880C991CAA1CBB1C8A95D1F746
:103EF000C701BE010E94692B6F01E12CF12CA701C3
:103F00009601260F371F411D511DC501B4010E94A6
:103F1000912B69017A01E0918600F0918700CA0136
:103F2000B9010E94592B9B01AC01DF010E94D72BE4
:103F30009B01AC01C701B6010E94592BDC01CB01EA
:103F40002FE0B695A795979587952A95D1F700917B
:103F500086001091870020E030E0081719072A0733
:103F60003B0728F46091860070918700CB01BC016B
:103F700070938B0060938A00DF91CF911F910F9116
:103F8000FF90EF90DF90CF90BF90AF909F908F9079
:103F9000089508950E94141F82E28093800089E1B1
:103FA000809381008FEF9FEF90938700809386002E
:103FB0000C94081E539A2BB1277F3BB138604FB742
:103FC000F894FC01CB01880F991F680F791F6E0FC1
:103FD0007F1FE617F70789F0819198E03BB9000051
:103FE00000C087FF2BB9880F000000C000C000C0D0
:103FF0002BB900C09A9591F7ECCF4FBF8FE594E0B5
:104000000197F1F700C000000895CF93DF93EC0112
:10401000FB018281882309F43CC1C430FDE5DF0740
:1040200060F4CB3F9CE5D90788F49E0122503C45C3
:104030002431310508F02EC109C0C236EDE5DE0796
:1040400029F0C63AFDE5DF0709F024C10E94340FCC
:104050009093C9028093C802C1318CE5D80709F456
:10406000C6C008F042C0C930ECE5DE0709F49BC0C9
:1040700000F5C5308CE5D80709F485C078F4C33065
:10408000ECE5DE0709F478C008F07AC0C230DC4500
:1040900009F0F5C08091C8028160EFC0C7309CE58F
:1040A000D90709F478C008F07AC08091C80280610D
:1040B000E4C0CD30FCE5DF0709F487C058F4CB300D
:1040C0009CE5D90709F479C008F07BC08091C8024B
:1040D00088606FC0CF30FCE5DF0709F480C008F0CE
:1040E00082C08091C802877FC8C0CE3F9CE5D907B7
:1040F00009F471C000F5C531FCE5DF0709F485C09E
:1041000068F4C3319CE5D90709F475C008F095C07F
:104110000E94E5088091C8028F77AFC0CC3FFCE5D4
:10412000DF07A9F108F054C0CB3FDC4509F0A7C078
:104130008091C90240C0C230EDE5DE0709F489C0B4
:1041400058F4C1158DE5D80709F45AC008F069C0C4
:104150008091C90282602FC0C236EDE5DE0709F406
:104160007CC0C63AFDE5DF0709F481C0C330DD45F8
:1041700009F085C080E06EC08091C80282607DC079
:104180008091C80216C08091C802886076C0809174
:10419000C90282604FC08091C80280626EC0809167
:1041A000C80280646AC00E94E5088091C8028068E5
:1041B00064C0846062C081603DC08091C8028E7F0F
:1041C0005CC08091C8028D7F58C08091C80216C023
:1041D0008091C90218C08091C9028D7F2BC0809147
:1041E000C8028F7E4AC08091C8028F7D46C08091F0
:1041F000C8028F7B42C08091C802877F8B7F3DC001
:104200008091C9028D7F8E7F15C08091C80282FB8C
:10421000222720F991E0922790FB82F990FB83F905
:104220002CC08091C902982F909591708E7F892B18
:1042300090FB81F98093C90222C00E94E508809119
:10424000C80287FB222720F991E0922790FB87F98B
:1042500014C081E00E94CB0F12C08091C80284FB81
:10426000222720F991E0922790FB84F906C08091E3
:10427000C802982F909590FB80F98093C802809196
:10428000C8029091C9020E94450F0E94E50880E093
:1042900001C081E0DF91CF910895CF93DF93863104
:1042A0009C4541F5EB010E94380E982F8A812091A0
:1042B000020130910301882379F09A7A81E009F4B0
:1042C00080E080939702911102C069E201C065E32A
:1042D000C9010E9443230AC080919702811102C044
:1042E00069E201C065E3C9010E944E230E947A0E73
:1042F00080E001C081E0DF91CF9108950F931F937B
:10430000CF93DF93C42FD22FFC0182818823C9F081
:1043100040939A020E9407249093990280939802F6
:1043200080E28C0F883008F057C0C77081E001C070
:10433000880FCA95EAF7DF91CF911F910F910C94E6
:10434000420680919A02481330C080919802909161
:1043500099020E941F24883C910538F510E21D0F38
:10436000CD17B9F080E28C0F883040F4C77081E03F
:1043700001C0880FCA95EAF70E944906183028F54F
:1043800081E09D2F977001C0880F9A95EAF70E94EF
:104390004206802F0E9439061830F0F4D77081E071
:1043A00001C0880FDA95EAF70AC080E28C0F8830E6
:1043B00098F4C77081E001C0880FCA95EAF7DF91D1
:1043C000CF911F910F910C944906802FDF91CF91CF
:1043D0001F910F910C943906DF91CF911F910F918E
:1043E00008950F939C01CB01243F4CE5340731F134
:1043F00088F4293DFCE53F07D9F02A3D4CE5340718
:1044000079F1283D3C45A9F506E221EE41EE68ED43
:104410007CE52BC0263FFCE53F07E1F0A8F0273FF5
:104420003C4539F507E225EE46EE67EF7CE51DC019
:1044300007E225EE45EE69ED7CE517C006E221EEC8
:1044400040EE64EF7CE511C007E225EE44EE65EF37
:104450007CE50BC006E221EE42EE66EF7CE505C08E
:1044600008E221E045EE6AED7CE50E947E2180E0D5
:1044700008C0FC018281882319F010929A0201C0C1
:1044800081E00F9108959093C5018093C401089530
:104490009093A00280939F020895E0919F02F09173
:1044A000A002309721F00190F081E02D099480E086
:1044B0000895E0919F02F091A002309799F0209129
:1044C0002B01222359F02091C80227FF07C0DC01ED
:1044D0002C9111962C93119726E02C930280F38156
:1044E000E02D09940895E0919F02F091A002309789
:1044F00039F022E0DC012C930480F581E02D099451
:10450000089520919D0230919E022817390771F07D
:1045100090939E0280939D02E0919F02F091A002F1
:10452000309721F00680F781E02D099408952091BD
:104530009B0230919C022817390771F090939C02DE
:1045400080939B02E0919F02F091A002309721F0AE
:104550000084F185E02D09940895FC013296809144
:104560002B01882331F08091C80287FF02C09EE1B1
:1045700001C096E080E0915028F021912223D9F3E8
:104580008F5FF9CF0895662351F120912B012223EB
:10459000E9F02091C80227FF19C0462F469546959D
:1045A00046954E31E0F4677021E030E002C0220F02
:1045B000331F6A95E2F7FC01E40FF11D828190E060
:1045C0002823392381E0232B69F409C0FC013296AA
:1045D00008962191621729F0E817F907D1F780E0D2
:1045E000089581E008959C01FC0132969FEF80E0E0
:1045F0004191461789F09F3F19F4411101C0982F4E
:104600008F5F8630A9F79F3F39F0F901E90FF11D5F
:1046100097FDFA956283089508959C012A5F3F4FA4
:10462000FC014281461301C0128201968217930752
:10463000B9F70895262F2695269526952E3168F4EC
:10464000FC01E20FF11D677021E030E001C0220F94
:104650006A95EAF78281282B22830895262F2695D2
:10466000269526952E3170F4FC01E20FF11D67703E
:1046700021E030E001C0220F6A95EAF7209582819F
:1046800028232283089520912B01222329F02091B1
:10469000C80227FD0C941A230C94F32220912B01BD
:1046A000222329F02091C80227FD0C942E230C947C
:1046B0000D2320912B01FC013296222331F08091B1
:1046C000C80287FF02C08EE101C086E0DF011D92B3
:1046D0008A95E9F7089508950C946B2383E08093FD
:1046E000A1020C946C23811102C081E001C082E020
:1046F0008093A1020C946C230C94732381E080932B
:10470000A1020C946C230C947E2308950C948523B1
:104710000C9486230C9485230C9485230C94852378
:10472000CF930E948C230E94D5130E948A23C0E05D
:104730008C2F0E94FF12892B29F4CF5FC430C1F760
:1047400080E001C081E0CF91089508951F920F92FB
:104750000FB60F9211248F939F93AF93BF938091C5
:10476000A202811113C08091EC029091ED02A09100
:10477000EE02B091EF024196A11DB11D8093EC02B3
:104780009093ED02A093EE02B093EF02BF91AF9130
:104790009F918F910F900FBE0F901F901895809151
:1047A000F402843031F10E9483041092A20220E4CA
:1047B00088E190E00FB6F894A895809360000FBE52
:1047C0002093600083B7817F846083BF83B781605B
:1047D00083BF7894889583B78E7F83BF0FB6F89494
:1047E000A8958091600088618093600010926000BD
:1047F0000FBE08950E94E5080C948A0482E084BDEF
:1048000093E095BD9AEF97BD80936E0008952FB702
:10481000F8948091EC029091ED02A091EE02B0919B
:10482000EF022FBF08952FB7F8946091EC027091BA
:10483000ED028091EE029091EF022FBF08959C014E
:104840004FB7F8948091EC029091ED02A091EE02A6
:10485000B091EF024FBF821B930B089578941F9283
:104860000F920FB60F9211248F939F93AF93BF9324
:104870008091EC029091ED02A091EE02B091EF02D6
:104880000196A11DB11D8093EC029093ED02A093BF
:10489000EE02B093EF02BF91AF919F918F910F9075
:1048A0000FBE0F901F90189581E08093E00080E28A
:1048B0008093D8001092C9008FE19EE40197F1F730
:1048C00000C0000087E090EBDC018093FD02909334
:1048D000FE02A093FF02B09300039CE088E10FB6B4
:1048E000F894A895809360000FBE90936000FFCF6E
:1048F0008091C6020895089522E02093E9002FEFE9
:104900003091E800215035FD06C035ED3A95F1F7BC
:1049100000002111F5CF2091E80025FF0BC040E0F9
:1049200050E066E070E00E94BB268091E8008E7740
:104930008093E8000895CF93DF9320912B012223E9
:1049400039F02091C80227FF03C060E222E002C0D4
:1049500068E021E02093E9002FEF3091E80021503A
:1049600035FD06C035ED3A95F1F700002111F5CF80
:104970002091E80025FF1DC0EC0180912B018111E1
:1049800005C040E050E068E070E003C070E040E047
:1049900050E0CE010E94BB268091E8008E77809384
:1049A000E80080E2FE01A6EAB2E001900D928A954D
:1049B000E1F7DF91CF9108958093A3027093A50250
:1049C0006093A4028091F402843001F582E0809328
:1049D000E9008FEF9091E800815095FD06C095EDBC
:1049E0009A95F1F700008111F5CF8091E80085FFDD
:1049F0000DC040E050E063E070E083EA92E00E9486
:104A0000BB268091E8008E778093E8000895BC0172
:104A100084E00C94DC24BC0183E00C94DC248091C1
:104A2000F302811109C00E944C280E94A92880919C
:104A3000E20084608093E20008951092F3020895EA
:104A40000C9483236091F00281E0611101C080E049
:104A50000C946E239091F40281E0943009F080E090
:104A60006091F0020C94732342E061EC81E00E94BB
:104A7000C52742E261EC82E00E94C5279091F402D2
:104A800081E0943009F080E06091F0020C947C2386
:104A90008091F602833009F461C030F4813071F006
:104AA000823009F49AC008958A3009F486C08B30A8
:104AB00009F46CC0893009F0A8C020C08091F502CB
:104AC000813A09F0A2C08091E800877F8093E800D6
:104AD0008091F9029091FA02892B21F460E286EA32
:104AE00092E003C060E080E090E070E00E94062762
:104AF0008091E8008B778093E80008958091F5021B
:104B0000813209F082C08091F9029091FA020297F5
:104B100008F07BC08091E800877F8093E800809157
:104B2000E80082FD05C08091F4028111F8CF6DC0CC
:104B30002091F3008091F20090E0922B029731F4E3
:104B40008091F100813011F0863021F48091F100E4
:104B50008093C6028091E8008B7753C08091F50264
:104B6000813A09F052C08091F9029091FA02892BA2
:104B700009F04BC08091E800877F8093E800809126
:104B8000E80080FFFCCF80912B0136C08091F502B8
:104B90008132D9F58091F9029091FA02892BA9F519
:104BA0008091E800877F8093E8000E94FA27809137
:104BB000F70280932B010C94E5088091F502813275
:104BC00021F58091E800877F8093E8000E94FA2712
:104BD0008091F8028093C70208958091F502813A8E
:104BE000A1F48091E800877F8093E8008091E8003D
:104BF00080FFFCCF8091C7028093F1008091E80094
:104C00008E778093E8000C94FA27089584B7877F05
:104C100084BF0FB6F894A895809160008861809356
:104C20006000109260000FBE90E080E80FB6F8942C
:104C300080936100909361000FBE0C947E230E94CC
:104C40004C280E94A928E2EEF0E0808184608083F5
:104C500078940C943E2B8FE191E00C944822809143
:104C6000F4028530A9F48091F402853079F40E9431
:104C7000CF238091F2028823B1F30E9490238823EE
:104C800091F30E94A5260E94E508EDCF0C94FA232B
:104C9000089508950C944C26292F3327233031058D
:104CA000C9F060F42130310581F02230310509F07E
:104CB00044C08BE390E025E934E043C02132310564
:104CC000E1F02232310549F138C082E190E020ED77
:104CD00034E037C099278130910549F028F00297D8
:104CE00061F5EFE6F4E005C0E1E9F4E002C0EDE7CC
:104CF000F4E0849190E09F0124C06115710541F0BA
:104D000061307105D1F489E090E020EC34E019C005
:104D100089E090E027EA34E014C06115710541F0A4
:104D20006130710551F486EB90E022EE34E009C069
:104D300080E490E028E935E004C080E090E020E0E5
:104D400030E0FA0131832083089580E189BD82E15A
:104D500089BD09B400FEFDCF8091D8008F7D80937E
:104D6000D8008091E00082608093E0008091E000B4
:104D700081FDFCCF0895CF92DF92EF92FF920F93C7
:104D80001F93CF93DF93EC018B017A010E941928C6
:104D9000811133C0E114F10439F0F7018081918170
:104DA000081B190BC80FD91FC12CD12C01151105D7
:104DB00019F18091E80085FD16C08091E8008E779A
:104DC0008093E800E114F10449F0F70180819181BA
:104DD000C80ED91ED182C08285E00FC00E9419285A
:104DE000882321F30AC089918093F10001501109B1
:104DF000FFEFCF1ADF0ADACF80E0DF91CF911F916A
:104E00000F91FF90EF90DF90CF9008952091FB02DB
:104E10003091FC022617370748F06115710539F407
:104E20002091E8002E772093E80001C0B901FC0131
:104E300020E06115710579F18091F4028823F1F188
:104E40008530F1F18091E80083FD3CC08091E8005D
:104E500082FD2EC08091E80080FFEBCF2091F3000F
:104E60008091F20090E0922B6115710551F088302D
:104E7000910538F421912093F10061507109019658
:104E8000F3CF21E0089709F020E08091E8008E77C9
:104E90008093E800CECF2111CFCF0AC08091F402D9
:104EA000882361F0853061F08091E80083FD0AC0BD
:104EB0008091E80082FFF2CF80E0089582E00895BB
:104EC00083E0089581E008952091FB023091FC0277
:104ED0002617370748F06115710539F42091E8006D
:104EE0002E772093E80001C0B901FC0120E0611594
:104EF000710591F18091F402882309F440C0853056
:104F000009F43FC08091E80083FD3DC08091E80036
:104F100082FD2FC08091E80080FFE9CF2091F3004F
:104F20008091F20090E0922B6115710559F0883064
:104F3000910540F424912093F1003196615071095C
:104F40000196F2CF21E0089709F020E08091E80077
:104F50008E778093E800CBCF2111CCCF0AC080910F
:104F6000F402882361F0853061F08091E80083FDD0
:104F70000AC08091E80082FFF2CF80E0089582E0CD
:104F8000089583E0089581E00895982F973068F59B
:104F90009093E900981739F07091EC002091ED00A2
:104FA0005091F00003C0242F762F50E021FD02C065
:104FB0009F5FECCF3091EB003E7F3093EB00309160
:104FC000ED003D7F3093ED003091EB003160309388
:104FD000EB007093EC002093ED005093F0002091D3
:104FE000EE0027FDE5CF80E008958F708093E90003
:104FF00081E008958091F50287FF11C08091E8005B
:1050000082FD05C08091F4028111F8CF11C080911A
:10501000E8008B770BC08091F402882349F08091DF
:10502000E80080FFF8CF8091E8008E778093E80059
:1050300008952091E4003091E50095E64091EC0060
:10504000842F817040FF23C08091E80080FD1DC047
:105050008091F402882399F0853099F08091EB00DB
:1050600085FD11C04091E4005091E50024173507FB
:1050700029F3915011F09A01E1CF84E0089582E084
:10508000089583E0089581E0089580E008954091B7
:10509000E80042FFDDCF08950E94BA280E94C2288E
:1050A000E0EEF0E0808181608083E8EDF0E08081D7
:1050B0008F77808319BCA7EDB0E08C918E7F8C93A5
:1050C00080818F7E80831092F30208950F931F9347
:1050D000CF93DF930E94BA280E94C228C8EDD0E087
:1050E00088818F77888388818068888388818F7D95
:1050F000888319BC1092F4021092F0021092F2020E
:105100001092F10200EE10E0F80180818B7F808325
:1051100088818160888342E060E080E00E94C5274A
:10512000E1EEF0E080818E7F8083E2EEF0E080812E
:1051300081608083808188608083F80180818E7F98
:105140008083888180618883DF91CF911F910F9147
:105150000895E8EDF0E080818F7E8083E7EDF0E058
:1051600080818160808384E082BF81E08093F3024C
:105170000C946628E8EDF0E080818E7F80831092A9
:10518000E20008951092DA001092E10008951F9253
:105190000F920FB60F9211242F933F934F935F936B
:1051A0006F937F938F939F93AF93BF93EF93FF93EF
:1051B0008091E10082FF0BC08091E20082FF07C076
:1051C0008091E1008B7F8093E1000E943D2B8091D4
:1051D000DA0080FF1FC08091D80080FF1BC0809143
:1051E000DA008E7F8093DA008091D90080FF0DC0B5
:1051F00080E189BD82E189BD09B400FEFDCF81E077
:105200008093F4020E940F2505C019BC1092F4028D
:105210000E941D258091E10080FF19C08091E2006D
:1052200080FF15C08091E2008E7F8093E200809124
:10523000E20080618093E2008091D80080628093D8
:10524000D80019BC85E08093F4020E942225809149
:10525000E10084FF30C08091E20084FF2CC080E137
:1052600089BD82E189BD09B400FEFDCF8091D800DF
:105270008F7D8093D8008091E1008F7E8093E10044
:105280008091E2008F7E8093E2008091E200816055
:105290008093E2008091F002882311F084E007C03F
:1052A0008091E30087FD02C081E001C083E080932C
:1052B000F4020E942A258091E10083FF29C0809199
:1052C000E20083FF25C08091E100877F8093E100A9
:1052D00082E08093F4021092F0028091E1008E7FD0
:1052E0008093E1008091E2008E7F8093E2008091C4
:1052F000E20080618093E20042E060E080E00E9492
:10530000C5278091F00088608093F0000E942025DE
:10531000FF91EF91BF91AF919F918F917F916F918D
:105320005F914F913F912F910F900FBE0F901F9063
:1053300018951F920F920FB60F9211242F933F933F
:105340004F935F936F937F938F939F93AF93BF938D
:10535000CF93DF93EF93FF93C091E900CF708091DB
:10536000EC00D82FD17080FDD0E81092E900809138
:10537000F000877F8093F00078940E94DD291092DE
:10538000E9008091F00088608093F000CD2BCF7011
:10539000C093E900FF91EF91DF91CF91BF91AF9161
:1053A0009F918F917F916F915F914F913F912F913D
:1053B0000F900FBE0F901F9018951F93CF93DF9300
:1053C000CDB7DEB7AA970FB6F894DEBF0FBECDBF3C
:1053D000E5EFF2E08091F100819322E0ED3FF207EA
:1053E000C9F70E9448258091E80083FF2EC1809173
:1053F000F5029091F602492F50E04A30510508F02D
:1054000024C1FA01EE59FF4F0C94B32B803821F0E0
:10541000823809F01AC108C08091F1029091F2021D
:10542000992389F082600FC08091F9028F708730D4
:1054300008F00BC18093E9008091EB0085FB882781
:1054400080F91092E9009091E800977F9093E8002E
:105450008093F1001092F100D1C0282F2D7F09F028
:10546000F4C0882319F0823061F0EFC08091F70218
:10547000813009F0EAC0933009F080E08093F202B5
:105480002EC08091F70281112AC08091F9028F709D
:105490002FEF280F263008F0D8C08093E900209124
:1054A000EB0020FF1CC0933021F48091EB00806260
:1054B00014C09091EB0090619093EB0021E030E0FC
:1054C000A90102C0440F551F8A95E2F74093EA00F4
:1054D0001092EA008091EB0088608093EB001092BC
:1054E000E9008091E800877F8093E8000E94FA2716
:1054F000ACC08111AAC01091F7021F778091E30020
:105500008078812B8093E3008091E800877F8093EF
:10551000E8000E94FA278091E80080FFFCCF80918C
:10552000E30080688093E300111102C082E001C0B3
:1055300083E08093F40289C08058823008F085C0EF
:105540008091F7029091F8028C3D53E0950779F530
:1055500083E08A838AE289834FB7F894DE01139649
:1055600020E03EE051E2E32FF0E050935700E49159
:1055700020FF03C0E295EF703F5FEF708E2F90E049
:10558000EA3010F0C79601C0C0968D939D932F5FAF
:10559000243149F74FBF8091E800877F8093E8006E
:1055A0006AE270E0CE0101960E94062716C0609163
:1055B000F9027091FA02AE014F5F5F4F0E944A26D6
:1055C000BC01892B09F441C09091E800977F90932A
:1055D000E80089819A810E9464278091E8008B7796
:1055E0008093E80032C0803881F58091E800877FA1
:1055F0008093E8008091F0028093F1008091E800B0
:105600008E7772CF811121C08091F7029091F802BC
:1056100099270297D4F48091E800877F8093E8006F
:105620008091F7028093F0020E94FA278091F002A5
:10563000811106C08091E30087FD02C081E001C0B6
:1056400084E08093F4020E9434258091E80083FF77
:105650000AC08091E800877F8093E8008091EB008A
:1056600080628093EB00AA960FB6F894DEBF0FBE5F
:10567000CDBFDF91CF911F9108950895CF93809171
:10568000F4028823A1F0C091E900CF709091EC0062
:10569000892F817090FD80E8C82B1092E9008091DD
:1056A000E80083FD0E94DD29CF70C093E900CF910F
:1056B0000895DB018F939F930E94D72BBF91AF91E9
:1056C000A29F800D911DA39F900DB29F900D11245C
:1056D0000895AA1BBB1B51E107C0AA1FBB1FA61739
:1056E000B70710F0A61BB70B881F991F5A95A9F78B
:1056F00080959095BC01CD01089597FB072E16F477
:10570000009407D077FD09D00E94692B07FC05D0D3
:105710003EF4909581959F4F0895709561957F4FC8
:105720000895A1E21A2EAA1BBB1BFD010DC0AA1FE2
:10573000BB1FEE1FFF1FA217B307E407F50720F0FA
:10574000A21BB30BE40BF50B661F771F881F991F75
:105750001A9469F760957095809590959B01AC01BE
:10576000BD01CF010895EE0FFF1F0590F491E02DCC
:1057700009940E94C12B332312F48A1B9B0B0C94B7
:10578000D22BA29FB001B39FC001A39F700D811DBA
:105790001124911DB29F700D811D1124911D08953A
:1057A0000E94C12BB7FF0895821B930B08950E949E
:1057B000C12BA59F900DB49F900DA49F800D911DAE
:1057C00011240895B7FF0C94D72B0E94D72B821B6E
:1057D000930B0895FC014150504030F001900616A3
:1057E000D1F73197CF010895882799270895FB01B4
:1057F000DC0104C08D910190801921F4415050408A
:10580000C8F7881B990B0895F999FECF92BD81BD09
:10581000F89A992780B50895A6E1B0E044E050E0F9
:105820000C943E2CA8E1B0E042E050E00C943E2CF9
:10583000262FF999FECF92BD81BDF89A019700B449
:10584000021639F01FBA20BD0FB6F894FA9AF99AE9
:105850000FBE08950396272F0E94192C0E94182C22
:10586000252F0E94192C242F0C94192C0196272FD8
:105870000E94192C0C94182CDC01CB01FC01F99925
:10588000FECF06C0F2BDE1BDF89A319600B40D928C
:0C58900041505040B8F70895F894FFCF45
:10589C00C8004802280850011E0A14010101020028
:1058AC000400040401191A1B1C1D1E1F2021227840
:1058BC00249B247C240B2507257B2401E200E90092
:1058CC00EA00B500B600B700CD008301CC008A0118
:1058DC0092019401210223022402250226022702AE
:1058EC002A02B300B4006F007000818283E200E9E9
:1058FC0000EA00B500B600B700CD008301CC008AE9
:10590C00019201940121022302240225022602277E
:10591C00022A02B300B4006F007000818283F1F0A0
:10592C00C6676630943137353497F4F5F6F70001D5
:10593C00020202020606060909090909090F0F0FDE
:10594C000F0F0F15151518191919191919191919E6
:04595C0019232400E7
:00000001FF
